:10000000831686011F308500831203109F0110287C
:1000100000009A0B0828051824289B0B08280800C4
:1000200001308600860D860D031818280820132835
:10003000860C860C031812280820192800009A0B39
:100040001E289B0B1E28080002309E00733086007D
:100050001E201E2086011E207C3086001E201E20B1
:1000600086011E209E0B262835288601051C352872
:1000700002309E000F3086001E201E20F0308600C9
:100080001E201E209E0B3A284B28820777343E34D0
:100090005E3406343F348601051C4B289D011D0843
:1000A000452086001E201E2086011E209D0A053048
:1000B0001D06031D4F28602800009A0B5C280800CD
:1000C000851C69281F18602806145C2006101F1460
:1000D00060281F108601051C60287228820773346F
:1000E0003F3478349D011D086E2086001E201E209E
:1000F00086011E209D0A03301D06031D7328A628B5
:1001000082073F3406345B344F3466346D347D34BB
:1001100007347F346F34403480309B009A0B8E2834
:100120009B0B8E28080020309A009A0B9528080017
:100130008C0186179320051E9F288C0A9A280C088C
:10014000802086008C2086138C20080098200518BB
:0E015000AA28A6281E200518AA281E2010285E
:02400E001F0091
:00000001FF
